:020000040000FA
:02000000FD28D9
:080008008131232923009D181A
:100010001D121D1620002208A6002308A700A80113
:10002000A901003200320000911A0F32FF30A807F8
:10003000A93DA63DA73D031C0800280FF333290F57
:10004000F2334230A800A901EE3323001908200042
:1000500003140800111EFE3323009A00200003142D
:100060000800230091002300950115141308910A3C
:100070000319920A20000800230093000430950021
:1000800055309600AA30960095149518FE33151138
:10009000910A0319920A20000800A900850122088C
:1000A00080388400230980058413A90803191E32AF
:1000B000F030AB0028088038AA00F030AB030319F9
:1000C000AB000319A9030319113200327A2003018E
:1000D00032182308A81F2308A80803190301AA0F30
:1000E00002328006E73300320000E733230884172A
:1000F00080040800330832040319B20A8030321A2F
:10010000B3063219B306B218B306330DB20DB30DF0
:1001100032080800A901A800FF30A807031CA9079E
:10012000031C08000330A700DF309820F533A70137
:10013000E83EA600A709FC30031C0332A6070318FB
:10014000FD33A6070000A70FF93326180032A61CBE
:100150000232000000320800003803191532AE00E8
:100160002608840027188317A701A601AE1B0832B2
:100170000008A600AE1C0832840A0008A70004325A
:10018000C5200005031DA60A080001302E180935F8
:10019000AE180935AE1809352E19090E0800AB0145
:1001A000AA011030AC00270DAA0DAB0D2808AA0239
:1001B0002908AB3B031805322808AA072908AB3DDC
:1001C0000310A60DA70DAC0BEE3326080800103067
:1001D000AF00A701A601AD0CAC0C031C043228082B
:1001E000A6072908A73DA70CA60CAB0CAA0CAF0BC1
:1001F000F2332A08080020000800230019309B0071
:1002000020309E0090309D002000A001220091012E
:1002100093010F3021009E0023008C018D013230AC
:1002200021008D006F308C0022009E019D0108305E
:1002300023009F008C012530210097006A3099002F
:1002400020008931AE292000D50803190232D503D8
:100250000132E617BD08031D0332BE08031906323A
:1002600001302000BD020030BE3B01326715B708E7
:10027000031D0332B8080319063201302000B7020B
:100280000030B83B01326714B508031D0332B608CD
:100290000319063201302000B5020030B63B0132AE
:1002A000E714D70803190232D7030132E717D80839
:1002B00003190232D803023268146812C308031DFE
:1002C0000332C4080319063201302000C302003093
:1002D000C43B0132E8160B1109008B132100951164
:1002E0001514951415159512200095018B168B1772
:1002F0000800661D043222008C1320000232220006
:100300008C1720006518023222008D13200008008F
:10031000661801320800661D043222008C17200086
:10032000023222008C1320000800E61C0432220056
:100330008D112000023222008D1522000D138D1325
:1003400020000800E51B01320800E61C04322200F0
:100350008D152000023222008D1120006616080043
:10036000813179218131952122000C122000080071
:1003700067136400C108031D0332C2080319053264
:1003800001302000C1020030C23B8C1A10326F08CD
:10039000C2006E08C100681F0A328B1F02328B1325
:1003A000FC334608C4004508C300E8128B17681FD9
:1003B0000632E81A04326F08C2006E08C10000302D
:1003C000E41B0130B40001308C1A0030B40503196D
:1003D0000232E514093203010D1A013E651A013A91
:1003E0000319E510031DE5146916E51C6912641E66
:1003F000053242084104031D0132E51065184232FE
:10040000E51C3F32DD08031D03326514E71639325F
:100410000030681A0130B4000030E8190130B4052A
:1004200003190432E001E716651402325D08E000AA
:10043000E00803190E32023080318A208C1A07320C
:10044000E81D05326816E71665140130E000E00388
:10045000EF33E81D0332681A0132080003010D1A58
:10046000013E651A013A03196510031D6514641EE7
:10047000053242084104031D01326510651C01323A
:10048000E7160432E51802326510671703018D1A6A
:10049000013EE51A013A0319E510031DE514E916BA
:1004A000E51CE912013065180030B4000130E41891
:1004B0000030B40503191332E41D0532420841042B
:1004C000031D0132E51065190532E51C0232E716FD
:1004D00065150432E518023265116717013265119E
:1004E000E71E0B32853156256A0835026B08363B0C
:1004F000031802328431F524E712671F0532843174
:10050000B72485310F25671303016518013E65196E
:1005100001380319E511031DE515E51D0432681EB8
:100520000232853146256911691E0132691508308C
:100530005F05A501A400083A2504031D01326915D1
:1005400010305F05A501A400103A2504031D0332F5
:10055000E91E0132691508006811E91C0132080022
:10056000C808031D0732C708031D0332671C013288
:100570006815193202304802031D0A32E71F07329C
:10058000E81C023268150332671C013268150B3211
:10059000043048020319043206304802031D0332B6
:1005A000671C0132681508000030661B0130B4007A
:1005B0000030E9190130B404031901320800813117
:1005C000B821893133218131A221813188295E0806
:1005D00080313120D600E0305605D900590E0F3950
:1005E000D900D936D1015908510203182C32E61628
:1005F000561CE612E61E03325B08CB0002325A0894
:10060000CB008B1F02328B13FC330D30A200013064
:10061000A3004908A8004B0880314D208B17C0016A
:10062000BF01C008031D0C323F085C02031C0832E6
:10063000053080318A200530BF070030C03DF133DE
:10064000D10AD636D0333732D101053080318A20F5
:100650008231D422D10A8C305102031DF6334E0868
:1006600080313120D100CE0A053080318A202F30F0
:100670005102031C0D323A305102031809325F3027
:100680005107B101B000B10D2F303002DE0012323F
:1006900041305102031C0D325B3051020318093204
:1006A0005F305107B101B000B10D36303002DE00CD
:1006B000013201328C33C001BF013F0839024008CA
:1006C0003A3B031C0A32053080318A208231D42221
:1006D0000530BF070030C03DF033D108031D123292
:1006E000C001BF013F083B0240083C3B031C0A32EB
:1006F000053080318A208231D4220530BF07003096
:10070000C03DF033510A031DAA3308008B1F02328B
:100710008B13FC33643080318A200630E3002100E3
:1007200026082000091E06328A31DF22691F0232A4
:100730005030E3000D30A2000130A3005408A8009F
:10074000630880314D20643080318A208B17080087
:1007500022000D138D132000D933D30153088031AB
:100760003120D100D30A510A031DF8335308CE00BB
:100770008331242385310F25C70108008131A2214F
:10078000813188214F30CE006617833124236613D0
:100790008131B021E51D02320F3201320800641DA3
:1007A00002328431F52C22008D130D1320006812C3
:1007B00022000C162000E2330030641A0130B4002D
:1007C0000030E4190130B404031905320B30A900DC
:1007D000B83080318B208131B82122008D130D1368
:1007E00064002000E51D06320C1B0232F433023295
:1007F0008431F52C22000C162000E4180232661415
:1008000001326610BB3308000C1F06328131B8215B
:10081000691901320800F8334D30D500E6130C1B7E
:1008200009328131B821691901320800E61F01320D
:100830000800F53308000F300C05E0006008A80040
:100840000F3C031C43322835A80784313424A6000A
:10085000A80A84313424A700A80A843134248031C2
:10086000AC202608E100323228080B000D34003499
:1008700000340134003400340234003400340334D2
:1008800000340034043400340034053400340034BF
:1008900006340034003407340034003408340034A3
:1008A00000340934003400340034003400340E3491
:1008B000003400340F34003400340A34003400347F
:1008C0000B34003400340C34003400340800671258
:1008D00084310C2469190132080084311B24610819
:1008E000CF008431042469190132080084311B24AB
:1008F0006108D0000C1F06328131B821691901321C
:100900000800F8334F0EF039CF0050084F04D100E3
:10091000671608006410E41069180132E4146411C9
:1009200008008B134E0823009100200051088031ED
:100930003C20CE0A84316724FF3051020318013273
:10094000671269190232FF30D1003E304E02883101
:1009500003191E284E082300910020005108803101
:100960003C20CE0A510A031DE53388311E2845304C
:1009700080313120E000A1306002031C0232A0303F
:10098000E000AD016008AC00A9016430A80080312E
:10099000E720BF002B08C0004008A7003F08A600C2
:1009A000A9014130A8008031CF20E0006008D500C7
:1009B000E6130800610880313120E0004730600212
:1009C000031C02324630E000AD016008AC00033089
:1009D000A9008B30A8008031E720BF002B08C000A1
:1009E0008B1F02328B13FC3308004430E10084314A
:1009F000DA244008B6003F08B5008B173608EB0034
:100A00003508EA00E71008004330E1008431DA24B9
:100A10004008B8003F08B7008B1767100800463041
:100A2000E1008431DA24E008031D0232E7110132CB
:100A3000E7154008BE003F08BD008B17671108008E
:100A40004130E1008431DA244008C4003F08C3008B
:100A50008B174008C6003F08C500E8120800403068
:100A600080313120D100E415511CE4116416D11CF1
:100A70006412E416511DE4126417D11D6413681743
:100A8000511E6813E417D11EE4130800473080316B
:100A90003120E000AD016008AC00A9010F30A800D2
:100AA0008031E720D8006810681608002E30D70083
:100AB000E71308003E3080313120CF0065174F1C0E
:100AC0006513E815CF1DE811E8174F1EE8136914E8
:100AD000CF1E6910E9144F1FE91006304F05C800FA
:100AE00008004E3080313120C9000800D108031DB4
:100AF000023284318A2401305102031D023264140F
:100B0000E41402305102031D0132E4140330510297
:100B1000031D0132641504305102031D1732661D96
:100B2000043222008C172000023222008C13200095
:100B30000130A900F43080318B20661D0432220080
:100B40008C132000023222008C1720000800423053
:100B5000230091002000510880313C205108DD0025
:100B60000800CE018431912CD3015308803131200B
:100B7000E000D30A600A031DF8335308CE00843125
:100B8000912CD108031D02320130D10043302300E3
:100B900091002000510880313C203633053051024D
:100BA000031802320530D1004E302300910020009E
:100BB000510880313C209533D108031D02320130A9
:100BC000D1004430230091002000510880313C289E
:100BD00080305102031807323E302300910020007C
:100BE000510880313C2020305105A501A400203A55
:100BF0002504031D0132E41008001A305102031CC1
:100C000002321930D10048302300910020005108F1
:100C100080313C205108DA005A355A07DB00AD011B
:100C20005A08AC00A9010A30A8008031E720DC0096
:100C3000AD015A08AC00A9011E30A8008031E720A0
:100C4000B9002B08BA00AD015A08AC00A901463022
:100C5000A8008031E720BB002B08BC00080045300D
:100C6000230091002000510880313C2846302300A9
:100C700091002000510880313C2820305102031897
:100C800009323F30230091002000510880313C2080
:100C90005108DF000800403051020318093240308B
:100CA000230091002000510880313C2085312F2500
:100CB00008004130230091002000510880313C2879
:100CC0004730230091002000510880313C285930E2
:100CD000230091002000510880313C28D108031DD9
:100CE00008325A30230091000030200080313C202F
:100CF00007325A30230091000130200080313C201F
:100D00000800D108031D08325B3023009100003039
:100D1000200080313C2007325B30230091000130FD
:100D2000200080313C200800D108031D08325C30CF
:100D3000230091000030200080313C2007325C30DD
:100D4000230091000130200080313C200800D108B0
:100D5000031D08325D3023009100003020008031F7
:100D60003C2007325D3023009100013020008031AB
:100D70003C200800D108031D08325E30230091009A
:100D80000030200080313C2007325E30230091008B
:100D90000130200080313C20080067120F300C0524
:100DA000E0000B3060020319013208008431042492
:100DB000E61F0132080069190132080008305F059A
:100DC000A501A400083A250403191E3201305F056D
:100DD000A501A40024032504031D043222008D175D
:100DE0002000023222008D13200002305F05A50191
:100DF000A400023A2504031D043222000D1720002E
:100E0000023222000D1320008131B821691901320C
:100E1000080084311B246108CC0049308031312026
:100E2000D2004C0852020319013208008431042414
:100E3000691901320800E61F0132080084311B24C1
:100E40006108CC004A3080313120D2004C08520277
:100E500003190132080084310424691901320800A1
:100E6000E61F0132080084311B246108CC004B309E
:100E700080313120D2004C0852020319013208009F
:100E80000C1F0132FD33E20184316724671A0132FD
:100E900008005108E20084316724671A0132080013
:100EA0008131B8216919013208008B1F02328B137E
:100EB000FC33E208031D033285317625BF32013051
:100EC0006202031D03328531E825B8320230620226
:100ED000031D033286313D26B13203306202031D09
:100EE000033286314B26AA3204306202031D0332DC
:100EF00086315926A33205306202031D0332853143
:100F0000A7259C3206306202031D03328531C125BC
:100F1000953207306202031D03328531DC258E32A3
:100F200008306202031D033286312F2687320930D2
:100F30006202031D03328631362680320A30620295
:100F4000031D03328631602679320B306202031DA5
:100F500003328531FD2572320C306202031D0332EB
:100F60008531B12D6B320D306202031D03328531A4
:100F7000B42D64320E306202031D033284318A24A0
:100F80005D3210306202031D03328531CE255632A8
:100F900011306202031D0332863167264F32123050
:100FA0006202031D033286316E264832133062021C
:100FB000031D033286318126413214306202031D43
:100FC00004322100A6162000393215306202031DBA
:100FD0000432210026172000313216306202031D30
:100FE0000932D108031D03328B31322302328B3197
:100FF0003723243217306202031D0932D108031D42
:1010000003328B313C2302328B31412317321830AB
:101010006202031D033286319426103219306202B7
:10102000031D03328631A72609321A306202031DDE
:1010300003328631BA2602328B1708008B1708302C
:101040005F05A501A400083A250403190932E51D2E
:1010500007328131B821E71C02328331CF23F733C5
:10106000671A01320800E6158931332110305F0517
:10107000A501A400103A2504031D08326614E915E1
:1010800081318821E5138131952102328131A221FC
:101090000130A900F43080318B205230CE00220084
:1010A0000C1620008331242322000C1220008131F1
:1010B000B021E911E6118831642001306202031D7C
:1010C000023284318A2408008431F5248431B72423
:1010D0008531042585310F2585315A2585317125C6
:1010E000853156258531462585312F2585312025A9
:1010F000423080313120DD003F3080313120DF004F
:101100004E3080313120C9005930803131202100EA
:10111000A0004830200080313120DA005A355A07CB
:10112000DB00AD015A08AC00A9010A30A8008031EB
:10113000E720DC00AD015A08AC00A9011E30A80070
:101140008031E720B9002B08BA00AD015A08AC0085
:10115000A9014630A8008031E720BB002B08BC0065
:101160005A30803131202100013903192611031D25
:1011700026155B3020008031312021000139031910
:10118000A611031DA6155C302000803131202100FE
:10119000013903192612031D26165D302000803107
:1011A0003120210001390319A613031DA6175E3053
:1011B0002000803131202100013903192910031D3D
:1011C0002914200008000030661A0130B4000030F5
:1011D00067180130B40403194532E6158231D42270
:1011E00022000C162000681D143221002608200061
:1011F00009190432CE0183312423073222000C1254
:1012000020008A31D0228B314623853104250130DC
:10121000C70004305F05A501A40025082404031DB0
:101220001D32003064190130B400013068190030FB
:10123000B405031904328331A82383318623013096
:10124000E4180030B400013069180030B404031908
:101250000432681902328331A823003222000C12B2
:101260002000E6110800641F1C328C1A19328531E7
:1012700056258C1A1632E71FFC338B1F02328B1354
:10128000FC33BF30B6007C30B500E7108B1722006E
:101290000C1620008331A8238331862322000C12F0
:1012A0002000651C243222000D132000641C033230
:1012B000E51366100800E51722008D172000E41CD6
:1012C000033266100800123266140030E41A01304E
:1012D000B40042084104031902320301031D013026
:1012E000B405031903326610813179213632651D48
:1012F0001632813179216610003064180130B40053
:101300000030E4180130B40403190332E5138131CD
:10131000B029E51722000D17200008001E32E61D37
:101320001C3222008D130D13200064181532E517AE
:1013300022000C1601302000E4180030B400003008
:10134000651B0130B405031903326614080003322B
:101350006610813179210132E513080066132100FE
:10136000A61226132000E9114C3080313120CF0025
:1013700065164F1C6512E516CF1CE5124D30803105
:101380003120CF00E6144F1CE6106615CF1C661105
:10139000553080313120EC00563080313120ED0065
:1013A000573080313120EE0080313320EF00813121
:1013B000B02181316D218831642084318A248131CA
:1013C000B821E51932328231AC22681D0632043070
:1013D0004802031902328831E320E51904328131D1
:1013E000B02185315625671D1932E71D1732E615E4
:1013F000893133218131A221210026082000891959
:1014000003328331AD2304328A31D5228B31462316
:1014100085310F25E51902328131B0210C1F0432CC
:10142000691D02328631CD26CA33651C03326C0831
:10143000D40002326D08D400E51D0332E814681CA4
:10144000E8108131B821E51D3932893133218131EC
:10145000A22181318821E71C02328331CF230C1F66
:101460000F328631CD26E5190B3222008D130D1374
:101470002000671E05321030E70685310F255732F0
:1014800085310F2500302100A61A01302000B4005C
:1014900000302100261B01302000B4040319023261
:1014A0008B31752304304802031D06328231AC2291
:1014B000681D02328831E320C433C53322000D1386
:1014C0008D132000651B15322100A1012100210888
:1014D0002002200003190B320A3080318A202100BB
:1014E000A10A20008131B821E5196933EF33813138
:1014F0007921C7018231AC228131B821E5195F33EE
:10150000E61FFA338831E32085314625E81F0E3285
:101510008131B821E5195333681AFA33043048028F
:10152000031D0432671468158831E320E810C201F6
:10153000C101E51902328131B021E513661066124E
:101540003E332100A20123001D121D162100230895
:10155000200080312A2023001E0820008918013233
:10156000FA3308000F302100A3002000EA330530D1
:101570002100A3002000E53306302100A300200055
:10158000E03307302100A3002000DB3308302100C6
:10159000A3002000D63301302100A3002000D13366
:1015A00002302100A3002000CC3303302100A3002F
:1015B0002000C73304302100A3002000C2332100E3
:1015C000A30120008A31A1220830A3009830A20094
:1015D00080310620031C03322100A400A40921004D
:1015E000240C200003186917031C69132100240C24
:1015F000890C20000318E917031CE913210083104C
:101600002419831420008318E917831CE9130800A8
:1016100009302100A30020008A31A1220130A3005B
:10162000F430A20080310620031C02322100A40005
:1016300021002408A700200008000A302100A30090
:1016400020008A31A1220130A300F430A2008031B1
:101650000620031C02322100A40021002408A80057
:10166000200008000B302100A30020006A330C305A
:101670002100A300200065330D302100A3002000CD
:1016800060330E302100A30020005B3385314625F6
:1016900023001D121D16200091120030911A0130F6
:1016A000B400003068180130B4040319F633003078
:1016B00068180130B4000130911A0030B4050319E4
:1016C00007320F3080312A202100A61420000800A4
:1016D000A301C830A20080310620031C0232210081
:1016E000A4002100A61420000800210026082000E4
:1016F000891E03328A31BC2202328A31C1228131F1
:10170000B821E519FC338A31B2222100A612261332
:0817100020000800FF33FF3345
:020000040001F9
:02000E009CCF85
:02001000FFDE11
:10E00000490057003000450041004300FF00540024
:10E01000450053005400FF00FF00FF00FF00FF0019
:10E02000FF00FF00FF00FF00FF00FF00FF00FF00F8
:10E03000FF00FF00FF00FF00FF00FF00FF00FF00E8
:10E04000FF00FF00FF00FF00FF00FF00FF00FF00D8
:10E05000FF00FF00FF00FF00FF00FF00FF00FF00C8
:10E06000FF00FF00FF00FF00FF00FF00FF00FF00B8
:10E07000FF00FF00FF00FF00FF00FF0000000000A6
:10E0800000000A000000010003000A0000000F0069
:10E0900005000400030000000300030073005400A7
:10E0A0004F00FF004F004B00FF0074006A00DC00CF
:10E0B0000500000001000000000000000000A900B1
:10E0C000BF00BE00BC00B800B000A000A100A300CB
:10E0D000A700AF004200810085006100200084009D
:10E0E0006300800040008E00650082004300410014
:10E0F000670086008B0062006000210064008800D9
:10E10000660089008D0083002000560065007200C3
:10E11000730069006F006E0020003900300030008D
:02E12000FF00FE
:00000001FF
